:030000000219FDE5
:03000B000200AA46
:03002B0002016669
:03005B000202FCA2
:030073000202E2A4
:1000800002030406080C10182030406080040608A3
:100090000C10182030406080A0C000070F1F3F0DDB
:1000A0000D0403060D0503030202C2AFC0D0C0E079
:1000B000206217E5256002E473E525F4F58A758B67
:1000C00000D262D0E0D0D0D2AF3285268AC262E5BB
:1000D00026F46036306803207210758B00D0E0D0B3
:1000E000D0C290C291C292D2AF32C290C291C2929B
:1000F000206E0D20660A7401D5E0FDE57EF4529075
:10010000758B00D0E0D0D0D2AF32758A00C28DD2CC
:1001100062210001B9306805206602D29001B93031
:100120006805206602D29101B9306805206602D2C6
:100130009201B9D29330680A2066077405D5E0FDB4
:10014000D29001B9D29430680A2066077405D5E0D0
:10015000FDD29101B9D29530680A2066077405D5A1
:10016000E0FDD29201B9C2AFC2AD53E6EFC0D0C03C
:10017000E0D2D3D2AFC2CEE52A6007207449152A57
:1001800021C77800790020742EE580307E01F4309C
:10019000E60278FF53DACF207E0343DA20307E0375
:1001A00043DA10C2D8C271E580307E01F430E60235
:1001B00079FFC3E89970CB306103752A402074033E
:1001C000752A40885FD27020740DE52B6004152BD2
:1001D00021D743DA01C2D820700221EAA85F20614A
:1001E00002C27020740221E888227882B604038556
:1001F0002224C3E52594404002D26420CF0AD0E0F7
:10020000D0D043E610D2AD32C2CF053A7802E52A0B
:100210006005307402152AC3E55F940140057562DC
:10022000004134756300756C00E5622401F562508D
:10023000037562FF7982B7020D306D1DC3E522940C
:10024000324016854D227982B7030E306D0BC3E51F
:100250002294324004798E8722C3E52395226008D8
:100260004004152341680523D8CA056CE56C70026B
:10027000156CD56D63756D017805C3E56C956E40A1
:1002800057C3E56C956F50087801756D0302029CA9
:10029000C3E56C957050057801756D01C3E56595F2
:1002A00024401E7982B7040241CD206D1485246557
:1002B000E56C046003856E6C756D0175233C02026C
:1002C000D8E5652850057565FF41CDF565E5650400
:1002D00070067563FF756CFFD0E0D0D043E610D296
:1002E000AD32C2AFC0D053E67FC260759100855673
:1002F00094855795759104D0D0D2AF32C2AF53E6F2
:10030000EFC2ADC0D0C0E0C0F0D2D3D2AFA8FBA93D
:10031000FCC2D8307102616353DACF207E0343DA26
:1003200010307E0343DA20D271E580307E01F42064
:10033000E602613A88278928A14253DACF207E035A
:1003400043DA20307E0343DA10C2D8C2713074021F
:10035000A12E7800E580307E01F430E602A12E88DF
:100360005FA11653DACF207E0343DA20307E0343A9
:10037000DA10C271206102813C53DACF207E034340
:10038000DA10307E0343DA20C2D8D271885A895BF2
:10039000C3E89558F8E99559F97B007E087A00C3BF
:1003A000E8948CE994005005755E00812E882178D0
:1003B000A2E6A8216055C3E894C8E994005008E477
:1003C000D2E4FB7A0A8109C3E89468E994015008F1
:1003D000E4D2E3FB7A0F8109C3E894D0E994025098
:1003E00008E4D2E2FB7A1E8109C3E894A0E99405EF
:1003F0005008E4D2E1FB7A3C8109C3E89498E9947F
:10040000085008E4D2E0FB7A787E00C3E8955CFCF3
:10041000E9955DFD30E70AECF42401FCEDF43400CD
:10042000FD755E00C3EC9AED9E5003755E01885C1D
:10043000895D855A58855B597802A116C3E89527CE
:10044000F8E99528F9307C0281FA307B0281FA3094
:100450007A0281F3207502815FE9FDE8FC817EE983
:10046000C313F9E813F830790281F3E9C313F9E80B
:0E04700013F830780281F3E9C313FDE813FCA2
:10047E00206126C3EC941CED940240028195ED7030
:10048E0018C3EC94C850120529C3E529940A5002EA
:10049E00A12E755F00D270A12EE529600215297478
:1004AE0000207F037896E624FAFEE43400FFC3ECC6
:1004BE009EFCED9FFD50067800790081FAC3EC9406
:1004CE00FFED9400400678FF790081FAEC8575F017
:1004DE00A4C5F0A2F733F87900400302051678FFA1
:1004EE007900020516E9C313F9E813F8307C0EE91A
:1004FE00600278FFC3E81338F8E43400F9C3E894D7
:10050E00FFE99400400278FF885FD270206102A15B
:10051E002E741FF4552F4BF52FC274EB7002D2744C
:10052E00752A40307403752A0A306102A142207484
:10053E000353DAFE207403752B20D0F0D0E0D0D018
:10054E00D2AD43E6103279010205727903020572CB
:10055E00790A020572791E020572796402057279B2
:10056E00C80205727817E4D5E0FDD8FAD9F6227ADA
:10057E00147B780205997A107B8C0205997A0D7B93
:10058E00B40205997A0B7BC80205997902B27DE413
:10059E00D294D5E0FDD291D5E0FDC291D5E0FDC259
:1005AE0094D5E0FDD290E576D5E0FDC2907496D557
:1005BE00E0FDD9D9EAF8D5E0FDD8FBDBCED2942206
:1005CE00C37C007D0075F00005F0EA33FAEB33FBD7
:1005DE0050F6EB13FBEA13FAC3E9FFE8FEE89AF8CC
:1005EE00E99BF95004EFF9EEF8B3EC33FCED33FD73
:1005FE00D5F0DFEDF9ECF822E889F08A20D2D4F8B4
:10060E00A9F07B0030F70B7BFFF42401F8E9F434FA
:10061E0000F9E88520F0A4ADF0F8E98520F0A4AF4C
:10062E00F0FEED2EF974003FFA7C04C3EA13FAE9EA
:10063E0013F9E813F8DCF48BF030F70AE8F4240130
:10064E00F8E9F43400F9E889F0C2D4F8A9F0227878
:10065E0082B604030206FCC3E55F9419401EE52D25
:10066E0054067018206D3678057994E71460077873
:10067E000A1460027812C3E54198401F306D098557
:10068E006765756CFF756D01852224E4F545F546A9
:10069E00F547F548F549C26D0206FCD26D7994E72F
:1006AE00147013E523F43333F913F8E9540104F904
:1006BE00E854FE0206F0E714147014E523F4333305
:1006CE0033F913F8E9540304F9E854FC0206F8E58B
:1006DE0023F433333333F913F8E954070404F9E8F8
:1006EE0054F8C39440F8E99400F98845894622C32A
:1006FE00E54113F9E54013F8C3E54598F8E5469949
:10070E00F9500CC3E89480E994FF4016020734C3F5
:10071E00E8947FE994005003020734787F79000251
:10072E000734788079FF884A894B22E54A2547F8B5
:10073E00E54B3548F9854B20E4300701F43549FA8D
:10074E0030E709C3EA94F04015020772C3EA940F2A
:10075E00500302077278FF79FF7A0F020772780052
:10076E0079007AF0C3E5249564500AC37401952488
:10077E00500B020790E54B20E70E020790E54B3039
:10078E00E706884789488A492278A4E6FAC3E54AEB
:10079E0033F8E54B33F9D106E930E70BC3E8948023
:1007AE00E994FF4013E1CAC3E8947FE99400500234
:1007BE00E1CA787F7900E1CA788079FFE820E715F1
:1007CE00C3E52398F84009C3E8940140030207F1FA
:1007DE0078010207F1E8F424012523F8400302070B
:1007EE00F178FF884C2278A5E6FAA848A949D106E7
:1007FE00E930E70CC3E89401E994FF40160208259E
:10080E00C3E894FFE99400500302082578FF7900AD
:10081E00020825780179FFE920E715C3E54C98F821
:10082E004009C3E89401400302084C780102084CC9
:10083E00E8F42401254CF8400302084C78FF882484
:10084E002278FFC26420693D206A12D264C3E5415A
:10085E00940A4009C3E52594405002C26479A1E789
:0F086E006023E541601F74FF8541F0848539F0F8
:10087D00306A0375F005A4F8C5F0600278FFC3E88F
:10088D0095675002A867886622C3E5409440E5410C
:10089D009401E56650031401A7046002F566227801
:1008AD0083E6F520120F4675E89012055475E89011
:1008BD00E5E820ECFBA8BDA9BE120FE075718075AF
:1008CD007202C3740213FD7480606613FC74802C75
:1008DD00FC74023DFDECFAEDFBC3E89AE99B401474
:1008ED00E5712480F571E5723402F572EA2CFAEBAC
:1008FD003DFB80E5AE71AF72C3E57213F9E571137F
:10090D00F8C3E913F9E813F87A03C3E913F9E81307
:10091D00F8DAF7AA201A70097571007572000209CC
:10092D003E1AEA6008EE28FEEF39FFDAF88E718F75
:10093D00722275E890227883E6FFE5E820ECF7A8AF
:10094D00BDA9BE0573C3E57394084052757300E9E4
:10095D00FA79A0E76044EA7007E574601B02097933
:10096D00C3E895746010E5745006600C1402098597
:10097D000460F9020985E574F574C394F6401B759E
:10098D0064C0C394064013756480C39406400B7510
:10099D006440C39406400375640075BB0E22EFC31B
:1009AD009401601F7480601BC3E894FFE9940350A9
:1009BD0012C3E89571E995725009E564600C1564F0
:1009CD000209D7E564F460020564A864C3E52498C0
:1009DD005002A824C3E89565400AA865E565F46052
:1009ED000385656488258826E573B4070375BB10F8
:1009FD0022743279A687F0A4C5F0A2F733F8C3E8C4
:100A0D0095644002A86488228824882588268867F2
:100A1D00227540007541F022C2AF75C820A8CCA93F
:100A2D00CDAA3A30CF010A75C824D2AFAB3BAC3C4E
:100A3D00883B893CC3E89BF8E99C206908F930673D
:100A4D0002613A4197AD3D8A3DF9EA9DFA6004781D
:100A5D00FF79FFAE3EAF3F8B3E8C3FC3EC9FFCC397
:100A6D00E99CF542A83BA93CC3E89EF8E99FF9C370
:100A7D00E54113FBE54013FAE82AF540E93BF54162
:100A8D0050067540FF7541FF41E1AA40AB41AC40B6
:100A9D00AD417E047F02C3EB940440021E1FC3EBE5
:100AAD00940840021E1FC3ED13FDEC13FCDEF7C3CB
:100ABD00EA9CFAEB9DFBEF6009C3E913F9E813F823
:100ACD00DFF7EA28FAEB39FB8A408B4150067BFFB2
:100ADD008B408B41C3EB94025002D2673069047F87
:100AED0003610C7892E6FFC3E537948240110FC382
:100AFD00E53794A040010FC3EF940640027F057EB9
:100B0D0004E541C4540FF9E541C454F0F8E540C47F
:100B1D00540F28F8C3E89EFAE99400FB4009C3EA94
:100B2D009402EB940050047A02E4FB6186AA40AB78
:100B3D0041EBC4FEEAC4540F4EFCC3EA9CFAEB949D
:100B4D0000FBC3E813C313F8EA28FAEB3400FB8A61
:100B5D00408B41C3EB94024002C2677804EBC4FEA4
:100B6D007B00EAC4540F4EFAC3EA98FA4005C394C9
:100B7D000250027A027892E6FF3060026186855259
:100B8D0056855357D26043E680C3E49AF8E49BF947
:100B9D003067028120E8FAE9FBD3E913FDE813FC85
:100BAD0088528953C3EF94036038EF20E00DE82C91
:100BBD00F8E93DF9ECFAEDFB020BDBE828F8E93931
:100BCD00F9C3E82402F8E93400F97AFE7BFFC3EF9C
:100BDD009403400E8A548B55884E894F8C508D51FD
:100BED008154885489558A4E8B4F8C508D51306964
:100BFD0020C3E53394034019E542A2E713F8E55508
:100C0D00F4240138400B20E7087554FFF42401F556
:100C1D00558154E8FAD3E813FC8852C3EF9403606E
:100C2D0020EF20E007E82CF8ECFA8140E8282402B8
:100C3D00F87AFEC3EF940340088A54884E8C508195
:100C4D005488548A4E8C50E56BC3335002646BF557
:100C5D006B306002815E753402D26043E680E52D13
:0F0C6D0054066026A840A941C3E913F9E813F81B
:100C7C00C2AF53E67F759100C3E498F594E499F5FF
:100C8C0095759104D26043E680D2AF22D26575444B
:100C9C0000752000306B03752040020CB7D26575CF
:100CAC004400752040306B03752000D2AF780120D2
:100CBC006722E52D54066002C265C3E541940540E8
:100CCC0013780294054008780394054002780630A6
:100CDC006902780A206019E544601530690AC3E599
:100CEC003394034003D53406D2AFD26CA1899166FC
:100CFC00D2AF0000C2AF206726E541C3FB940F4082
:100D0C00027B0FEB240530730123306A0274282018
:100D1C00620123F93069027982E58BC39940B505EC
:100D2C0044E59BF45440B52002A17330690A08C312
:100D3C00E8940A40010881E020650281B7C265533E
:100D4C00E67F7591003067107594007595FE75916E
:100D5C0004D26043E68081B7AE40AF41C3E49EF558
:100D6C0094E49FF595A15AC3E5339402500281B7E0
:100D7C0030650281B7D802A18781E0C26C53E67F4F
:100D8C00759100855494855595759104854E5685BD
:100D9C004F57D26043E680D2AFE52D540660082051
:100DAC006A020533020DC3306C0D206B0A206507F7
:100DBC001581158102161822780030640530650201
:100DCC007801E53775F007A4F9E5F028F5F0E9A20C
:100DDC00F013A2F113A2F213F537C39478500375F4
:100DEC003778C3E53795384008D266C290C291C2B5
:100DFC0092306002A1FD855056855157D26043E672
:100E0C008022207D11C2AF754302D294C293D2AF1F
:100E1C00759F11020FDDC2AF754302D294C295D2F9
:100E2C00AF759F11020FDD307243207D20C2AF756C
:100E3C004303900144757E10C292D295306204D265
:100E4C0091C151C294D2AF759F01020FDDC2AF7533
:100E5C004303900144757E10C290D293306204D249
:100E6C0091C171C294D2AF759F21020FDD207D1705
:100E7C00C2AF75430390011FC292306202D291D26D
:100E8C00AF759F01020FDDC2AF75430390011FC206
:100E9C0090306202D291D2AF759F21020FDD207D7E
:100EAC0011C2AF754304D293C295D2AF759F210284
:100EBC000FDDC2AF754304D295C293D2AF759F01BB
:100ECC00020FDD307243207D20C2AF7543059001C7
:100EDC0033757E08C291D294306204D290C1EDC2B7
:100EEC0093D2AF759F11020FDDC2AF754305900110
:100EFC0055757E20C291D294306204D292E10DC21B
:100F0C0095D2AF759F11020FDD207D17C2AF7543CF
:100F1C0005900115C291306202D290D2AF759F112B
:100F2C00020FDDC2AF754305900129C2913062EB0F
:100F3C00D292D2AF759F11020FDD207D11C2AF7519
:100F4C004306D295C294D2AF759F01020FDDC2AF9A
:100F5C00754306D293C294D2AF759F21020FDD3038
:100F6C007242207D20C2AF754301900155757E20E1
:100F7C00C290D293306204D292E189C295D2AF75FD
:100F8C009F21020FDDC2AF754301900133757E08BE
:100F9C00C292D295306204D290E1A9C293D2AF75BD
:100FAC009F01E1DD207D16C2AF754301900129C27E
:100FBC0090306202D292D2AF759F21E1DDC2AF7543
:100FCC004301900115C292306202D290D2AF759F4C
:100FDC0001C26622900113757E00C290C291C2922A
:100FEC00D293D294D295C262227880760708760783
:100FFC000876010876040876FF0876FF08760B0859
:10100C007602087601087601788C7601087600085D
:10101C0076B40876FF0876FF0876FF087603087624
:10102C00FF0876010876FF0876250876D0087678D2
:10103C000876C80876040876FF087601087600085A
:10104C00767A087607087601087601087600087625
:10105C00FF227887E6FFC272BF0302D2727888C281
:0F106C007DE630E102D27DC27E7889E630E10276
:10107B00D27EC3EF94026008758E01D2730210907A
:10108B00758E00C273227880E6149000809378A44A
:10109B00F67881E6149000809378A5F67886E614AE
:1010AB0090008D9378A6F6789FE6F8700108C3E858
:1010BB00941140027811E82828F56E256E256E28CC
:1010CB00F56F256E2828F570789CE67538FF753915
:1010DB000CB402067538A075390AB403067538824C
:1010EB0075390578A3E61490009A93F569120FE011
:1010FB0022227896E6FA7897E6FB7888E6B4030521
:10110B00C3EB940EFB307F047A007BFFC3EB9AFC9E
:10111B00C3948250027C827575000575EC8575F061
:10112B00A4C3E5F0947D40F222D27F11FD1205633A
:10113B007A007B007C10120559E55F2AFA74003B9C
:10114B00FBDCF37C04C3EB13FBEA13FADCF7FEC204
:10115B007F11FD22E5EF20E6037520000520903F6F
:10116B00FFE520146006901DFF14600093046003DC
:10117B0075EF1053D9BF7581C043FF8012055475AD
:10118B00EF0043B203E5B3240420E70DF521E5E3BB
:10119B0020E0068521B343E301120FE07580FF7554
:1011AB00A40075F1D075D4BF75907875A53F75F215
:1011BB00BF75D54075A60175E241E4F8F6D8FD750B
:1011CB006B01120FF512166078988676753001C296
:1011DB00AF12056D12057D120563120584120563AE
:1011EB0012058B12056312178312056D12056D1212
:1011FB000568C2AF78FA79FA308607D9FBD8F702BF
:10120B001C00115E119111FC11FD78988676120F5E
:10121B00E075885075891275C82475910475D8408E
:10122B0075A82275B80275E690759B80759D007543
:10123B00D10775BC5875BB0E75BA1175E8801205D0
:10124B0054D2AF1208AC53DACF207E0343DA2030EE
:10125B007E0343DA1043DA01C2D8C27112056DD294
:10126B00617B037A0CE55E70077A0CDB030211FDE0
:10127B001205632070030211FDC270E55FC3940277
:10128B0040E1E52F541F856160F561B560D5DAD576
:10129B00C26153DACF207E0343DA20307E0343DA78
:1012AB0010C2D8C27178A2E67008D274E52F54E050
:1012BB00F52FC275752900120568307409C3E5292D
:1012CB00940A4002D27512055978023074027800E4
:1012DB00C3E55F9840F0C2AF12057D12057D120584
:1012EB007DD2AF12056D754D00120559788CE6C392
:1012FB00940150030213CAE530C394015003021347
:10130B00CA207435C3E55F94FF50030213CAC2AF02
:10131B00120592D2AF120568C3E55F940150EFC27C
:10132B00AF12057D12055E12057DD2AF120568C3A3
:10133B00E55F94FF40E90218087F05D27F11FD128B
:10134B000568C2AFC27F11FDAE5FC3E55F947FD26C
:10135B00AF4076120554C2AF120592D2AFDFDC312B
:10136B0034C3EE94057897F612056D1216A2121778
:10137B008B7F0AD27F11FD120568C2AFC27F11FDB0
:10138B00AE5FC3E55F947FD2AF50E6120554C2AF98
:10139B0012057D12055E12057DD2AFDFD63134EE1C
:1013AB0024057896F612056D1216A21217BA1205BD
:1013BB006811FDC3E55F94FF5002610C021808C36E
:1013CB00E55F954D4003855F4D120568780179887F
:1013DB00E7B403027805C3E55F98400241F4C2AF5E
:1013EB00120592120592120592D2AF12056D75304D
:1013FB0000E4F531F5320531E531F4703905327819
:10140B009AE67819146012783214600D787D1460A6
:10141B000878FA146003753200C3E532984017154B
:10142B00327531B478998676C2AF120592D2AF7805
:10143B0098867612056812055EE52A7005307402EF
:10144B0021FD78012074027806C3E55F9840A7124E
:10145B000568E52A70030211FDC2AF120FE0E4F537
:0F146B0022F523F524F525F526F56AD2AF78850D
:10147A00E6C333F568E4F545F546F547F548F54919
:10148A00F573F52CF52DF53775730875BB10120534
:10149A005412093FE5E820ECFBA8BDA9BEE970019A
:1014AA00F8887412094375730875BB107887E6FECD
:1014BA007602115E7887EEF6C2AF7564FF1209FEF6
:1014CA00852264852265852266D2AF75220175243C
:1014DA000175250175260185636C756D017888E6AD
:1014EA00B40307C27D307602D27DD268D2697533E1
:1014FA0000120F46120F6B120A1E120A25120A1E3A
:10150A00120A25120A1E02151FC2AF115ED2AF754A
:10151A00730075BB0E120CA912065D120DC4120ED1
:10152A000E120A25120C98306D031206FD2067036D
:10153A0012084F306703120896120DC4120E3312A6
:10154A000A25120CA9306D03120739120DC4120EA6
:10155A00AA120A25120C98306D03120797120DC4AD
:10156A00120ECF120A25120CA9306D031207F412BB
:10157A000DC4120F46120A2512093F120C98120DB9
:10158A00C4120F6B120943120A2530692F206B2CE3
:10159A0085676485676585636C756D0179187A0C52
:1015AA00C3E533994009C269D26A8A350215C6C3AE
:1015BA00E55F9401400302151F021620306A1B20C2
:1015CA006B18E535147004C26AA113F535C3E55FDB
:1015DA009401400302151F021620753600C3E56206
:1015EA009401400985676585636C756D01C3E56281
:1015FA0078FA985021307404E52A601A78F0306B32
:10160A00058567647820C3E541985002A11F053615
:10161A00E55F6002C123753600C2AF120FE078871A
:10162A00E6FE7602115E7887EEF6E4F522F523F5FA
:10163A0024F525F526F568C268D2AF120554120FB3
:10164A00E0307406E52A700221FD788DE6C3940124
:10165A00400241D161FC901A0D78201216E4E5206F
:10166A00B4A50CA31216E4E520B45A03021682129A
:10167A000FF51216A20216A1901A0378807B0A129D
:10168A0016E4A308DBF9901A0F788C7B181216E47B
:10169A00A308DBF9901A2722C2AF1217231216FDEC
:1016AA00901A00740E1216E9A374041216E9A374B0
:1016BA00141216E9901A0378807B0A1216E8A30816
:1016CA00DBF9901A0F788C7B181216E8A308DBF95D
:1016DA00121736121714901A2722E493F622E643B9
:1016EA008F01538FFD75EF0275B7A575B7F1F053EA
:1016FA008FFE22438F02438F0175EF0275B7A575DE
:10170A00B7F1901A0DF0538FFC22901A0D74A5D1DF
:10171A00E9901A0E745AD1E9227A3079D078209059
:10172A001A40D1E4E520F709A3DAF7227A3079D012
:10173A00901A40E7D1E909A3DAF922AB77A878BB76
:10174A0001027980BB02027981BB03027982BB0460
:10175A00027994BB05027983BB06027986BB07022C
:10176A007992BB08027987BB0902799CBB0A027984
:10177A0088BB0B027989E8F7227C0512056DDCFB30
:10178A0022C2AF12057D12058412058B1205921230
:10179A00055E12057D12058412058B12059212054B
:1017AA005E12057D12058412058B120592D2AF22B4
:1017BA00C2AF12059212058B12058412057D12051D
:1017CA005E12059212058B12058412057D12055EC2
:1017DA0012059212058B12058412057DD2AF22AE34
:1017EA0077AF78C2AF12057D12057D12057D12050D
:1017FA005EDEF212059212055EDFF8D2AF221217F0
:10180A008B12178312178375770175780175790022
:10181A001217E97C05AD5F12056DC3ED955F70F592
:10182A00C3E55F9401400AC3E55F94FF403702189D
:10183A004C1217451216A212178BC2AF75EF10126F
:10184A001783DCD10579C3E5799403500280C1126C
:10185A0017830578E5771490009F93F808C3E57815
:0E186A0098500280A81217831217830577C3C7
:10187800E577940C50028094120FF51216A2C2AFAD
:0618880075EF101217833A
:0319FD0002115F75
:101A00000E041407070104FFFF0B020101A55A0190
:101A100000B4FFFFFF03FF01FF25D078C804FF01DA
:081A200000FF07010100FFFFB8
:101A40002344503341232020202020202020202008
:101A500023424C48454C4923463333302320202031
:101A60002020202020202020202020202020202076
:101C0000C2AFC2D353D9BF7581C043B20343FF8073
:101C1000752438752503B1C975EF0275E24043F1AB
:101C20004053A4BF75D400D2867DFA780379E67C50
:101C300010752200752300901DD67B0675249875BB
:101C400025013086028142208608D8FBD9F9DCF7CD
:101C500081B4308608D8FBD9F9DCF781B4B189E4C6
:101C600093A3C39A6004DDC381B4DBDBB17B600264
:101C7000812B7B08E493FAA3B15CDBF87A30B15C8A
:101C8000752200752300B17BEAFCEBFDC3ED94FEE9
:101C9000400EB17B8A278B28ED30E0048A828B834B
:101CA000B17B7AC270D8C3ED94FE601350CEBD00F4
:101CB00025EC60097520007521FF0200008100A855
:101CC00027A9280809D804D90281D3B17FEA89AAB3
:101CD000F281C50D81A0C3ED94035049EDA2E092BD
:101CE000007AC5C3E5829400E583941C50902000DF
:101CF00010438F02438F0175B7A575B7F1F030001F
:101D00001FA827A9280809438F01538FFDD804D99C
:101D100002A12089AAE275B7A575B7F1F0A3A10DBC
:101D2000538FFC817C7AC1BD030CE493A3FAB140CC
:101D3000DCF8B138817C817EAA22AB23B15CEBFA5E
:101D4000EA6222752608C3E52313F523E52213F57D
:101D50002250066323A0632201D526EAB1C9B1C986
:101D600075260AEAF4200102D286300102C286B149
:101D7000C9C3134002C201D526EB22B17FEAFB2082
:101D80008602A17F308602A184752608AE24AF2585
:101D9000C3EF13FFEE13FEB1CDB1C9C3EA13308612
:101DA000024480FA30E703632201C3E52313F523DD
:101DB000E52213F52250066323A0632201D526D91C
:101DC000E52265236523F52222AE24AF250E0FDE22
:101DD000FEDFFCD20122424C48656C693437316326
:041DE000F3300601D5
:00000001FF
